:100000000C944A030C9482030C9482030C94820394
:100010000C9482030C9482030C9482030C9482034C
:100020000C9482030C9482030C9482030C94CF29C9
:100030000C947E2A0C949F240C9482030C948203CB
:100040000C9482030C9482030C9482030C94282554
:100050000C9482030C9482030C9482030C9482030C
:100060000C9482030C9482030C9482030C948203FC
:100070000C9482037C077C07A807A80716081009C0
:100080001009100934089C08AD08AD08E31BE61BF5
:10009000EB1BF21BF71BFC1B011C061C0B1C101C92
:1000A000151C1A1C1C1C1F1C221C251C281C2B1C6C
:1000B0002D1C301C341CBD1DC01DEA1DFD1D051E60
:1000C000101E131E131E131E5B1E5B1E181E1B1E0E
:1000D000201E2D1E3A1E3D1E411E4E1EBC1E2E1FF2
:1000E000C41E8E1E921EC81E951ECB1ED61EA01E9E
:1000F000241FA41EDA1EA81EDE1E081FAC1EE21E50
:10010000121FB21EE81EF21E991ECF1E9C1ED21E8A
:10011000B71EED1EFE1E1E1F201F8A1EC01E371F8B
:100120007323792367236D237F2385238B23E62A7B
:100130000D2B052C0D2B052C592B7C2B052CD32B93
:10014000E22B290014001A000800150017001C00FB
:1001500018000C00120013002B21040016000700E9
:1001600009000A000B000D000E000F002800E1003E
:100170001D001B00060019000500110010003600CC
:10018000370038432921E200E3002C412C42E700EC
:10019000E600E400000000002A0035021E021F02F3
:1001A0002002210222022302240225022602270223
:1001B0000100010001000100010001002D022E02DA
:1001C0002F02300231020100010001000100010094
:1001D0000100010033003400520001000100010061
:1001E000010001000100500051004F00000000001C
:1001F0004C0035001E001F002000210022002300BB
:1002000024002500260027003A003B003C003D006A
:100210003E003F002D002E002F0030003100400036
:1002200041004200430044004500320064000100E8
:1002300001000100010001000100010001000100B6
:1002400001000100000000004C00A8003A003B0043
:100250003C003D003E003F004000410042004300A2
:1002600001000278057804781570207823781470DE
:100270002578277845003900007C0678037801004E
:10028000217824780100267828780100A600010052
:100290000100010001000100010001000000000058
:1002A00044001E0F0500047F3F1F643214643214A3
:1002B000783C1E1E140A052223252628292A2C2DC7
:1002C0002F3032333536383A3B3D3E404243454786
:1002D000494A4C4E5051535557595A5C5E606264BE
:1002E0006668696B6D6F71737577797B7D7F8183CC
:1002F0008587898A8C8E90929496989A9C9E9FA1CD
:10030000A3A5A7A8AAACAEAFB1B3B4B6B8B9BBBCED
:10031000BEBFC1C2C3C5C6C7C9CACBCCCDCED0D162
:10032000D2D2D3D4D5D6D7D7D8D9D9DADADBDBDB5A
:10033000DCDCDCDCDCDDDDDDDDDCDCDCDCDCDBDBFB
:10034000DBDADAD9D9D8D7D7D6D5D4D3D2D2D1D04F
:10035000CECDCCCBCAC9C7C6C5C3C2C1BFBEBCBB4C
:10036000B9B8B6B4B3B1AFAEACAAA8A7A5A3A19FC4
:100370009E9C9A98969492908E8C8A898785838188
:100380007F7D7B79777573716F6D6B696866646269
:10039000605E5C5A5957555351504E4C4A49474537
:1003A0004342403E3D3B3A3836353332302F2D2CD8
:1003B0002A292826252322FFAA7F55400001010172
:1003C0000101010101010202020202020202020312
:1003D00003030303030303040404040404040505E2
:1003E00005050506060606060707070707080808A5
:1003F00008090909090A0A0A0B0B0B0C0C0C0D0D54
:100400000D0E0E0E0F0F0F101011111112121313EB
:100410001414151516161717181819191A1A1B1B64
:100420001C1D1D1E1E1F20202122222324242526C0
:1004300026272829292A2B2C2D2D2E2F30313232F8
:10044000333435363738393A3B3C3D3E3F40414204
:10045000434445464748494A4C4D4E4F50515354EA
:10046000555658595A5B5D5E5F616264656668699E
:100470006B6C6D6F7072737577787A7B7D7E80821E
:10048000838587888A8C8E8F91939596989A9C9E67
:10049000A0A2A3A5A7A9ABADAFB1B3B5B7BABCBE77
:1004A000C0C2C4C6C9CBCDCFD1D4D6D8DBDDDFE244
:1004B000E4E7E9EBEEF0F3F5F8FAFDFF00000000E9
:1004C000000000002A2B28000000000000000000AF
:1004D0000000000000000029000000002C1E342055
:1004E000212224342627252E362D3738271E1F207B
:1004F0002122232425263333362E37381F040506C0
:100500000708090A0B0C0D0E0F1011121314151603
:100510001718191A1B1C1D2F3130232D3504050601
:100520000708090A0B0C0D0E0F10111213141516E3
:100530001718191A1B1C1D2F3130354C00000000F4
:1005400000000000000000000000000000000000AB
:10055000000000000000000000000000000000009B
:100560007E0F00D4FFFFFFC700000078100341009A
:100570004C004500540048003400320000000E03D7
:10058000320035004B0045005900530000000403C1
:10059000090409025B00030100A0FA09040000013C
:1005A000030101000921110100012240000705811A
:1005B00003080001090401000203000000092111E1
:1005C0000100012222000705820320000107050324
:1005D00003200001090402000103000000092111A9
:1005E00001000122320007058403200001120100EE
:1005F0000200000008D804C8EA0000010200010659
:1006000060FF0961A1010962150026FF00952075B0
:100610000881020963150026FF00952075089102E4
:10062000C005010980A101850319012AB700150140
:1006300026B700950175108100C0050C0901A101C4
:10064000850419012AA002150126A0029501751042
:100650008100C005010906A101050719E029E71578
:100660000025019508750181029501750881010534
:1006700007190029FF150026FF009506750881005F
:100680000508190129059505750191029501750364
:100690009101C00011241FBECFEFD4E0DEBFCDBF5B
:1006A00004B603FE18C08091EF029091F002A09171
:1006B000F102B091F2028730904BA740B04B59F451
:1006C0001092EF021092F0021092F1021092F202D8
:1006D000E0E0F8E3099511E0A0E0B1E0E0EFFBE530
:1006E00002C005900D92AA3EB107D9F722E0AAEE0A
:1006F000B1E001C01D92AF3EB207E1F70E946C1459
:100700000C94F62D0C940000CF93C62F811128C0B5
:10071000809104020E947405823059F08330D1F038
:10072000811127C0CC2311F08BE221C08BE292E033
:100730000AC08091B502CC2349F082FD02C081E954
:1007400016C085E394E00E94600413C082FDF9CFD7
:1007500080E90DC0CC2311F089EA09C08AEA07C0FC
:10076000813039F4662311F08EE401C08BE40E94DD
:100770002B0781E0CF91089584E00895282F8430DD
:10078000E8F46430D8F44B30C8F4862F90E06BE086
:1007900070E00E943C2CFC01822F90E06CE270E043
:1007A0000E943C2C8E0F9F1FFC01E40FF11DEE0FE9
:1007B000FF1FEE5BFE4F85919491089580E090E0DD
:1007C00008959C013A9521153F4130F5BC016627FB
:1007D0007270AC01442754709C012227387094FF3A
:1007E0000FC090FF02C080E101C080E0672B09F0DC
:1007F0008062452B09F08064232B79F0806808958E
:10080000892F8170672B09F08260452B09F0846085
:10081000232B19F08860089580E00895CF93DF932B
:10082000EB010E94E103FE010995DF91CF9108954C
:10083000CF93DF93EC01805E9109089710F0209729
:1008400019F465E377E002C069E779E0CE010E9420
:100850000E048C2F0E941106DF91CF910895CF9343
:10086000DF93EC010E94B206CE01805E91090897E9
:1008700010F0209719F46CE377E002C060E879E0AB
:10088000CE010E940E04DF91CF9108950F931F9324
:10089000CF93DF938C01EB010E941804209741F065
:1008A0008FE99FE00197F1F700C000002197F6CF94
:1008B000C8010E942F04DF91CF911F910F910895DD
:1008C0008933910519F060E070E002C060E570E0E6
:1008D0000E944604089581E0089581E008950E94F1
:1008E0006D04089508950E9472040895A5E0B0E093
:1008F000ECE7F4E00C94E62C49835A833091F10143
:1009000089819A81311114C0662359F0222349F05C
:100910000E94D80A182F682F89819A810E94AF0AF5
:1009200003C00E94C40A182F69817A81812F04C0F4
:100930000E94D80A69817A810E94EC112596E3E031
:100940000C94022DFC01262F40815181628173811C
:1009500084810E947604089581E00895CF93DF9307
:10096000EC0160E00E94A204BE010E947304DF91CA
:10097000CF910895E1E0F0E0DF0102C0AA0FBB1FB4
:100980006A95E2F7BD01DF0102C0AA0FBB1F4A95BD
:10099000E2F7AD01462B01C0EE0F2A95EAF7942F3E
:1009A0009823491302C08E2B0895E0958E23089555
:1009B000242F462F682F809104020E94BA040E94BF
:1009C000110A08950E94301308950E942A13089571
:1009D00008950E949D090E94E8042FEF84E39CE0A3
:1009E000215080409040E1F700C0000008950E942F
:1009F000E9040E944E2508950E94E9040E94722590
:100A000008950F931F93CF93DF938C0161E00E94B1
:100A1000A204EC01B8010E94D81C882309F450C03C
:100A2000B801CE010E946F04882309F449C0B801BF
:100A3000CE010E945B23882309F442C0B801CE0195
:100A40000E94661E8823E1F1B801CE010E94C122F6
:100A50008823B1F1B801CE010E94CD1B882381F11A
:100A6000F8018281882341F1C3308CE7D807D1F0A7
:100A700040F4C115FCE7DF0791F0C130DC47A1F07D
:100A80001BC0CB35ECE7DE07A9F0CC35FCE7DF0770
:100A900071F0CA35DC4781F40E94490F0DC00E94F5
:100AA000F7040EC00E94510F0E94FC0409C00E946E
:100AB0003F0F02C00E944D0FC8010E946B0401C08D
:100AC00080E0DF91CF911F910F9108950E947D24C6
:100AD0000E94A8050E94271A08950E94AC050E9452
:100AE000081B0E9486240895982F92959F7019F0F4
:100AF000892F24E001C020E0982F9695969511F05B
:100B00002E5F892F982F969509F02F5F822F0895D9
:100B100008950E948805089581E008950895CF936F
:100B2000DF93D82F0E948C05C82F882319F08D2FB2
:100B30000E948E058C2FDF91CF9108950895CF9359
:100B4000C82F0E9489058C2F0E948F05CF91089590
:100B500080E00E949F0508950E94A8230E949F059F
:100B60000895CF930E94A823C82F8091EC01C81745
:100B700079F0C093EC010E940D256093ED01709314
:100B8000EE018093EF019093F0018C2F0E949F055E
:100B9000CF910895ABE0B0E0E0EDF5E00C94E72CE8
:100BA0004F83588769877A878B8761110E94870EE8
:100BB0009E012F5F3F4F86E0F90111928A95E9F778
:100BC00085E0FE013796D90101900D928A95E1F7F3
:100BD00089819A814C815D81452B31F09F3F31F4B1
:100BE00091E08F3F19F403C091E001C090E090FFC5
:100BF00009C049815A816B817C818D819E810E94CF
:100C0000AC0D05C0C9010E94AC048111F2CF2B9636
:100C1000E2E00C94032DFC01808191810E94050B80
:100C20000895CF93882309F49BC0C82F8238C1F45C
:100C30000E94A82381FD94C069E3809104019091F2
:100C400005010E944C240E94AB0E2FEF87EE93E02B
:100C5000215080409040E1F700C0000069E319C0D6
:100C6000833801F50E94A82380FD7AC063E5809156
:100C70000401909105010E944C240E94AB0E2FEFBD
:100C800081EE94E0215080409040E1F700C00000E8
:100C900063E580910401909105010E944F240E9418
:100CA000AB0E5EC08438C1F40E94A82382FD58C0F8
:100CB00067E480910401909105010E944C240E94F8
:100CC000AB0E2FEF81EE94E0215080409040E1F791
:100CD00000C0000067E4DDCF8CEF8C0F813AD0F4C8
:100CE0006C2F80910401909105010E9416248823A5
:100CF00049F06C2F80910401909105010E944F24CE
:100D00000E94AB0E6C2F80910401909105010E940E
:100D10004C24C5CF80E28C0F883048F4C77081E046
:100D200001C0880FCA95EAF70E946A0EB8CFEBE5BA
:100D3000EC0FE33040F4F0E0EC5AFE4F808190E09D
:100D40000E94C0230DC0C85AC93150F4EC2FF0E006
:100D5000EE0FFF1FEE5DFE4F808191810E94E52323
:100D6000CF910895882309F45DC0682F823879F403
:100D70000E94A82381FF56C069E3809104019091ED
:100D800005010E944C240E94AB0E69E310C0833819
:100D9000B9F40E94A82380FF45C063E58091040157
:100DA000909105010E944C240E94AB0E63E5809156
:100DB0000401909105010E944F240E94AB0E0895FA
:100DC000843879F40E94A82382FF2CC067E48091C4
:100DD0000401909105010E944C240E94AB0E67E42F
:100DE000E6CF8CEF860F813A10F380E2860F8830D1
:100DF00048F4677081E001C0880F6A95EAF70E94A5
:100E0000700EDBCF8BE5860F833028F480E090E016
:100E10000E94C0230895685A693120F480E090E070
:100E20000E94E52308951F93CF93DF93182FEB01C2
:100E30000E941106209741F08FE99FE00197F1F79A
:100E400000C000002197F6CF812F0E94B206DF91EB
:100E5000CF911F910895893319F060E070E002C0CE
:100E600060E570E00E9413070895882321F00E9436
:100E70006A0E0E94AB0E0895882321F00E94700E26
:100E80000E94AB0E0895A0E0B0E0E9E4F7E00C9416
:100E9000E12C7C01162FC72FFC01D2810581029520
:100EA0000F700E94600E8823B9F0DD23A9F08C2F0B
:100EB000807F803421F080E2810F883068F080915B
:100EC000B60282FF09C082E00E940D0F0E94600EF0
:100ED00091E0D82ED92601C0D12CCC2EC2948FE01F
:100EE000C8228C2D90E08C30910508F099C1FC014E
:100EF000E65CFF4F0C94CA2C8C2F807FCF70882328
:100F000011F0C295C07FDD2399F0CC2309F474C1A0
:100F100080E2810F883010F0111104C08C2F0E94E4
:100F20006A0E03C08C2F0E947A0E0E94AB0E64C121
:100F3000812F0E94B206CC2309F472C180E2810F96
:100F4000883038F1112329F18C2F0E94800E24C0A3
:100F50008C2F807FCF70803211F0C295C07F11231B
:100F600019F01130D1F143C08091B60282FD17C053
:100F7000DD2349F0CC2329F08C2F0E946A0E0E94B9
:100F8000AB0E80E03AC180E00E94B206CC2309F4A7
:100F900047C18C2F0E94700E0E94AB0E41C1DD2311
:100FA00071F0002341F0013031F40E948A0E8C2B45
:100FB0000E94940E35C10E948A0E8C2B23C0011111
:100FC00003C00E94A10E2EC0013009F429C18C2F4C
:100FD0000E943C070E94A10E23C1DD2321F00630B0
:100FE00008F01EC10EC0053008F01AC11BC0DD2379
:100FF00061F0002331F0F701858180FFFDC08F7023
:1010000085838C2F0E9435070BC1002359F01933BB
:1010100009F003C1FFEF27EE83E0F150204080404C
:10102000E1F7F9C08C2F0E943C07FAC08C2F8695FF
:101030008695837019F0813061F0F2C0DD2321F0D4
:10104000812F9C2F937002C080E090E00E94C0230B
:10105000EFC0DD2321F0812F9C2F937002C080E030
:1010600090E00E94E523E4C08C2F837079F5D111C4
:10107000DBC0412F429546954770440F440F212F06
:101080002F70042E01C0220F0A94EAF714FF08C043
:101090008FE090E001C0880F4A95EAF7809501C083
:1010A00080E0C695C695C370822BC23049F058F4D3
:1010B000C13019F00E94020AB7C00E94FC09B4C0F6
:1010C0000E94080AB1C00E94F909AEC0DD2319F0E0
:1010D0008C2F817001C08695882309F4A5C0412F0B
:1010E000429546954770440F440F212F2F70042ED0
:1010F00001C0220F0A94EAF714FF08C08FE090E0C5
:1011000001C0880F4A95EAF7809501C080E0C69536
:10111000C695C370822BC23049F058F4C13019F023
:101120000E944E0A81C00E94480A7EC00E94540A52
:101130007BC00E94110A78C0CF70DD2339F08C2F5C
:101140000E94230A812F0E9435076EC0812F0E94C2
:101150003C078C2F0E942F0A67C0123F21F128F410
:10116000103F41F0113FC1F043C0133F19F1143F4C
:1011700079F03EC0DD2341F0053008F051C08C2FDE
:101180008F710E943C0A4CC0063008F049C0F7CF6E
:101190008091B60282FD18C0DD2339F08C2F8F714B
:1011A0000E94230A3DC0DD23C9F38C2F8F710E945A
:1011B0002F0A36C0DD2329F08C2F8F710E941A0A66
:1011C0002FC00E94160A2CC0DD2349F0CF718C2F4E
:1011D0000E94230A63E08C2F0E94EF0E21C081E061
:1011E0000E940D0F0230E0F082E00E940D0F18C047
:1011F000DD2331F0002391F2812F0E94110610C0EF
:10120000002399F2193349F49FEFE7EEF3E0915090
:10121000E040F040E1F700C00000812F0E94B206DC
:1012200088EF8C0D843020F40E94A8230E949F0533
:10123000DD2089F00E945C0E80FD0DC0F701128256
:101240000E94560E0E94230AC7010E9448090E946C
:10125000560E0E942F0ACDB7DEB7E8E00C94FD2CA5
:101260000F931F93CF93DF93EC01688179818A817B
:101270000E94100B8C010E945A0A0E94EC09B801CE
:10128000CE010E944307DF91CF911F910F910895E6
:10129000CF93DF93EC01988189812B813C81232BB3
:1012A00031F08F3F31F481E09F3F19F403C081E0BA
:1012B00001C080E080FD1AC0CE010E9401058111AD
:1012C0000FC00E94600E882389F08A81882371F004
:1012D0008091B60282FF0AC082E00E940D0F06C014
:1012E000CE010E943009CE010E94AE04DF91CF9161
:1012F0000895882321F00E947A0E0E94AB0E089573
:10130000882321F00E94800E0E94AB0E089580E099
:1013100090E00E94C02380E090E00E94E5230E94BC
:10132000870E0E94AB0E08958091040190910501F3
:101330000E9452240E94870908950E94770E0E94FD
:101340009409089592959F70963079F010F4925018
:1013500001C09A50923068F4803F69F018F4883EDA
:1013600040F409C0843F29F406C0883E20F0813F44
:1013700011F080E0089581E00895FC019081818161
:1013800023813481232B31F08F3F31F481E09F3F63
:1013900019F403C081E001C080E080FD07C08081B6
:1013A00091810E94050B0E94A209089580E0089592
:1013B000A5E0B0E0EEEDF9E00C94E72C2596E2E034
:1013C0000C94032DA6E0B0E0E8EEF9E00C94E72CD5
:1013D0002696E2E00C94032D089508950E94ED09ED
:1013E00008950E94EE0908950E94F1098093050274
:1013F00008950E94F409089590910502892B0E9496
:10140000F40908959091050289230E94F409089532
:101410009091050289270E94F40908950E94ED0920
:1014200008950E940E0A80930402089580E00E94AD
:10143000110A089591E001C0990F8A95EAF7892F62
:101440000E94110A089521E030E001C0220F8A9520
:10145000EAF780910402822B0E94110A089521E08C
:1014600030E001C0220F8A95EAF7209580910402AE
:1014700082230E94110A089521E030E001C0220F6A
:101480008A95EAF78091040282270E94110A089542
:1014900090910402892B0E94110A089590910402F0
:1014A00089230E94110A08959091040289270E94BD
:1014B000110A08950895282FFA01862F8770A1E058
:1014C00001C0AA0F8A95EAF7CB0133E0969587957C
:1014D0003A95E1F763E070E00E943C2CE80FF91FB9
:1014E00040E050E0622F70E090819B01042E02C02A
:1014F000369527950A94E2F72170219529272A230A
:10150000292721934F5F5F4F4330510569F70895B5
:10151000FB01A82FA77023E0969587952A95E1F700
:1015200063E070E00E943C2CE80FF91F40E050E0BF
:1015300080E0219130E00A2E02C0369527950A946A
:10154000E2F721703327042E01C0220F0A94EAF734
:10155000822B4F5F5F4F4330510559F70895943008
:1015600090F48B3080F4362F282F892F90E06BE099
:1015700070E00E943C2CBC01620F711D42EF51E0F3
:10158000832F0E945B0A0895943080F48B3070F4AE
:10159000282F892F90E06BE070E00E943C2C62EFD6
:1015A00071E0820F911D0E94880A089580E00895DD
:1015B000CF92DF92FF920F931F93CF93DF936C0133
:1015C0000091040280910502082BC7E0D0E010E0F2
:1015D000C8010C2E02C0959587950A94E2F780FD0C
:1015E00004C02197A8F7F12C07C0FC2EB6018C2F60
:1015F0000E94F8110197A9F38F2DDF91CF911F91D0
:101600000F91FF90DF90CF900895CF93DF93EC017F
:101610000E94D80ABE010E94F811DF91CF9108956F
:101620001F93CF93DF93EB019091F101992321F068
:10163000CB010E94050B13C0882349F0CB010E9407
:10164000D80A182F682FCE010E94AF0A04C0CB0120
:101650000E94C40A182FBE01812F0E94F811DF9149
:10166000CF911F910895CF93DF93C091060280918F
:101670000702C817A1F0D0E0CE0166E070E00E943A
:101680003C2CFC01E85FFD4F4081518162817381F8
:10169000848195810E94E2092196C770E8CFDF918D
:1016A000CF910895409138025091390260913A02E9
:1016B00070913B0280913C0290913D020E94E209B0
:1016C0000895CF93B82FC62F20910602A09107024C
:1016D0002A17B1F030E0C90166E070E00E943C2CAE
:1016E000FC01E85FFD4F81818C1306C080818B1364
:1016F00003C08281841306C02F5F3F4F2770E8CF5D
:1017000080E001C081E0CF9108951F93CF93DF93D4
:1017100080913D0282958F7009F05AC080913A0203
:10172000882309F455C02091060210910702C09148
:101730003802D0913902A0913B02B0913C0281E085
:10174000CF3F09F080E0482F211709F441C01097DE
:1017500021F0DF3F21F080E003C081E001C0842F51
:1017600030E080FD31C0C90166E070E00E943C2C91
:10177000FC01E85FFD4F81818D1326C080818C13B1
:1017800023C08281811120C0838194818A1B9B0B9D
:10179000883C9105C8F480913D028F7080618093F0
:1017A0003D02C90166E070E00E943C2CFC01E35F51
:1017B000FD4F90819F709061908388E392E00E943A
:1017C00048090E94330B04C02F5F3F4F2770BCCFE6
:1017D000DF91CF911F910895A1E1B0E0E2EFFBE02E
:1017E0000C94DD2C8C0185E0F801DE011D96019042
:1017F0000D928A95E1F7D8011296EC9090913802FB
:101800002091390240913B0250913C024115510513
:1018100031F02F3F31F481E09F3F19F403C081E0A4
:1018200001C080E080FD79C1F801C080D180838053
:10183000948088E3A82E82E0B82EF0903A02B4019A
:10184000641B750BFF2009F412C180913D02382FF3
:10185000307F683C710508F0CCC031118BC0D212CA
:1018600014C0C91212C0FE2CE1100FC08F7080612D
:1018700080933D020E94520BC5010E94480980914D
:101880003D02D80115968C9362C18114910439F000
:10189000BFEFDB1206C081E0CB1203C003C081E0C2
:1018A00001C080E080FD03C081E08E2502C080E0A1
:1018B00090E080FF10C04E2D6D2D8C2D0E94610B8D
:1018C000882349F088E392E00E944809E8E3F2E0C7
:1018D00086E0DF019EC08114910439F0BFEFDB1276
:1018E00006C081E0CB1203C003C081E001C080E0EC
:1018F00080FD03C081E08E2502C080E090E0E82FEB
:10190000E170BE2E80FF2CC04E2D6D2D8C2D0E94BF
:10191000610BF82E811124C0CD86DE868D859E85D3
:101920000E94050B292F22952F70223018F02430A9
:1019300090F405C09F7059F0811109C008C19F70D3
:1019400031F0D80115969C91907F09F400C1805E1A
:10195000883008F4FCC0C8010E944809FB2CF7C07D
:10196000FE2CEE2009F4F3C080913D02816080934B
:101970003D0254C0D21206C0C91204C0E11002C018
:10198000F80199C0C8010E94BD09882361F1EE20C9
:1019900051F120913D02822F82958F7090E0029745
:1019A00074F0809138029091390298878F8319865C
:1019B0009B868A862C87CE0107960E94480986E07E
:1019C000F801A8E3B2E001900D928A95E1F70E9438
:1019D000850B0E94520B0AC0D21611F1C8010E9459
:1019E000BD0981112CC0C8010E944809FF24F3944D
:1019F000AEC03111F1CF782D998A888AA6016E2D5B
:101A000089890E94D80988E392E00E94480986E00B
:101A1000D5011D928A95E9F70E94520BF12C97C0CF
:101A2000C912DCCFE110DACFF8018583C8010E942A
:101A3000480986E0D5011D928A95E9F788C0EE2015
:101A400091F220913D02822F82958F7090E0029753
:101A50000CF4B5CF80913802909139029A83898332
:101A60001B829D828C822E83CE010196A6CF683C7C
:101A7000710508F044C0FE2CEE2009F4B4CFD21258
:101A800030C0C9122EC020913D0220FD21C0822FFE
:101A900082958F70482F50E041155105C9F0F8012B
:101AA00025834F30510541F08F5F982F9295907F9D
:101AB000822F8F70892B8583C8010E94480986E098
:101AC000F801A8E3B2E001900D928A95E1F73DC0DC
:101AD00086E0F801A8E3B2E001900D928A95E1F763
:101AE00036C0C8010E94BD09811169CF80913D02B5
:101AF000816080933D02C8010E94480928C0782D6A
:101B0000998A888AA6016E2D89890E94D80986E063
:101B1000D5011D928A95E9F718C0EE2009F463CF2C
:101B2000C8010E94BD09F82E882309F45CCF86E025
:101B3000F801A8E3B2E001900D928A95E1F788E3FD
:101B400092E00E940B060E94850B0E94520B8F2D83
:101B50006196ECE00C94F92CACE0B0E0E2EBFDE037
:101B60000C94E72C4F83588769877A878B879C87EB
:101B7000CE0107960E94EC0B8823D1F09F818885C7
:101B80002A853B85232B31F08F3F31F481E09F3F45
:101B900019F403C081E001C080E080FD6FC04F8177
:101BA000588569857A858B859C850E94E20966C087
:101BB00086E0FE013796DE01119601900D928A951E
:101BC000E1F7FF81E8856A857B856115710531F054
:101BD000EF3F31F481E0FF3F19F403C081E001C021
:101BE00080E080FD4BC08091070290E09C012F5F58
:101BF0003F4F277033274091060250E024173507E6
:101C000009F443C0F983EA837D836C8366E070E066
:101C10000E943C2CDC01A85FBD4F96E0FE0131968E
:101C200001900D929A95E1F7209307020E94330BE1
:101C300025C090E066E070E00E943C2C885F9D4FDC
:101C40000E94EC0B882371F18091060290E066E01F
:101C500070E00E943C2CFC01E85FFD4F4081518107
:101C600062817381848195810E94E20980910602DC
:101C700090E0019687709927809306028091060272
:101C8000909107028913D5CF0DC00E949D09109233
:101C9000070210920602E8E3F2E086E0DF011D92FF
:101CA0008A95E9F72C96E2E00C94032D8091460288
:101CB000859585958595089580914602877008954C
:101CC00090914602977081E009F480E00895809138
:101CD0005102089590915102892B809351020895E9
:101CE000809590915102892380935102089510921A
:101CF0005102089590915002892B809350020895CB
:101D000080959091500289238093500208951092FB
:101D10005002089580914702089508950E948D0E03
:101D200008950E948E0E08959091B60292FF08C009
:101D300090914702981721F0809347020E94910EDC
:101D4000089580914702882329F01092470280E08D
:101D50000E94910E0895CF93DF93E0910401F091DA
:101D60000501809151028083E0910401F091050109
:101D7000908180915002892B808380914702882333
:101D800081F0E0910401F09105019081892B80831D
:101D900080910401909105010E940A2481110E9402
:101DA000A10EC0910401D091050148E050E06EE31E
:101DB00072E0CE010E94792D892B59F088E0FE0156
:101DC000AEE3B2E001900D928A95E1F7CE010E9458
:101DD000B523DF91CF9108950E948D0E08959091C3
:101DE000B60292FF11C0982F990F990F990F692B86
:101DF000609346020E94230A80914602859585954C
:101E000085950E94EC0E08950E94230A0895109271
:101E1000460280E00E94EC0E0895209146028095D3
:101E2000822380934602982F977099F430E0482FD0
:101E3000082E000C550B2417350759F09091B60267
:101E400092FF07C08595859585950E942F0A0E946F
:101E5000070F08959091B60292FB222720F92817C8
:101E600069F080FB92F99093B6028091B50290914F
:101E7000B6020E94730F82E00E940D0F08958091B8
:101E8000B60282FB882780F991E089270E942A0FF9
:101E9000089581E00E942A0F089580E00E942A0F91
:101EA00008956FEF7FEF80E090E00E94C12D0895CC
:101EB00080E090E00E949D2D873E9E4F19F40E9485
:101EC0006A1C089580E0089582E090E00E948F2DC2
:101ED000089583E090E00E948F2D089584E090E0C3
:101EE0000E949D2D0895BC0184E090E00E94C12DC8
:101EF0000895AB01BC018FE090E00E94B52D0895DC
:101F0000AB01BC0183E190E00E94B52D089560E033
:101F100070E0CB010E94800F089560E070E0CB017B
:101F20000E94790F0E94870F089567EE7EEF80E090
:101F300090E00E94C12D60E082E090E00E94A32D1D
:101F400060E083E090E00E94A32D1092050260E023
:101F500074E184E090E00E94C12D60E086E090E0B2
:101F60000E94A32D6FEF87E090E00E94A32D40E038
:101F700050E0BA0188E090E00E94B52D60E08DE06D
:101F800090E00E94A32D40E050E0BA0188E190E08B
:101F90000E94B52D60E087E190E00E94A32D40E013
:101FA00050E0BA018CE190E00E94B52D60E070E055
:101FB00080E290E00E94C12D40E050E0BA0188E14B
:101FC00090E00E94B52D80E00E94831C0E94B81C06
:101FD0000E948D0F08950E94950F0895682F8EE03E
:101FE00090E00E94A32D08950E940D256093640245
:101FF000709365028093660290936702609360021B
:1020000070936102809362029093630208950E942C
:102010000D2560936402709365028093660290932D
:10202000670260935C0270935D0280935E029093FE
:102030005F02089581E008950E941A10089508959E
:102040000E941F1008950E941F1008950E942310DF
:1020500008950E941F1008950E94291008950E945B
:102060001F1008958CED92E10E949E230E942F1074
:102070000E942C1008950E9420100E941F100895A5
:102080000E94F8120E949E0508950E94F8240E9462
:10209000C81C0E941B200E94D1130E9440100E9465
:1020A000C21A0E9426100895AAE0B0E0EAE5F0E125
:1020B0000C94DC2C0E94E71324E5E22E22E0F22EA1
:1020C0005701D12CF501019111915F018D2D0E94D5
:1020D000131380279127D394F4E0DF1619F0892B8E
:1020E00089F322C0892B01F50E9401258C01809182
:1020F0005202909153020817190709F45BC08FEF41
:1021000089838A831B820E9401258160782F9D83A9
:102110008C8349815A816B818D810E94CA051093FD
:1021200053020093520246C08091680281FD0E94D2
:102130001C130E941C10782E10E0812F0E94131394
:102140004C01F701A080B180A826B926A114B104E2
:1021500049F100E0CC24C394D12CC5018C219D21F0
:10216000892BC1F07720B1F00E831F8321E0C401D9
:102170008C219D21892B09F420E028870E940125CC
:102180008160782F9A8789874E815F8168858A85EB
:102190000E94CA050F5FCC0CDD1C0B30F1F6F70175
:1021A000918280821F5FF2E0EF0EF11C143029F65D
:1021B0000E94F40F0E94121B0E94922081110E9423
:1021C00007100E94B1052A96EDE00C94F82CCF93ED
:1021D000DF930E94FD11EC01811520E59207E0F5E7
:1021E000811530E4930708F09FC0803E910528F5E3
:1021F0008D3C910508F096C0883A910570F4853AB7
:10220000910508F085C08130910509F47EC008F47D
:10221000DCC0049708F0DCC0D8C0813C910508F010
:10222000D4C0C85AD0E0CC0FDD1FC95ADE4F099088
:10223000D881C02DCE019464CCC0C11580E2D807EE
:1022400008F0B8C0C11591E0D90708F0C1C0C83E78
:10225000D10508F4BDC0B9C0803622E5920738F533
:10226000803432E5930708F06CC0C03282E5D807AD
:1022700008F05EC0C11592E5D90708F48AC04C2F5A
:102280004695469550E0F5E0440F551FFA95E1F765
:10229000C37021E030E0C90102C0880F991FCA95C0
:1022A000E2F7EA01C82BD92BCE019D6892C0803A93
:1022B00022E59207C0F48F71C03832E5D30708F0E9
:1022C00056C08695869590E065E0880F991F6A95BF
:1022D000E1F7C37021E030E002C0220F331FCA953E
:1022E000E2F73A6841C0C03C82E5D80708F446C02E
:1022F000C03E92E5D90708F068C0CF71DD27DC2F1A
:10230000CC27CE01806F906A64C081E090E061C00C
:10231000C55AD0E0C757DE4F8881C82FD0E0CE0124
:10232000906457C0906555C0DF70CE01906A51C06F
:10233000CF718C2F90E0D82FCC27CE01816F906A7F
:1023400048C08F718695869590E09C0175E0220FBC
:10235000331F7A95E1F7C37081E090E002C0880FE7
:10236000991FCA95E2F79C68822B932B32C090E0AC
:10237000D82FCC27CE01846F906A2BC08C2F8F7101
:102380000E9499128F7190E0D82FCC27CE019062D5
:1023900020C08C2F8F710E94991295E0D695C79519
:1023A0009A95E1F7CF70D0E0DC2FCC27D0699E0161
:1023B000282B09C08D2F8F710E949912DD27D062C2
:1023C0008F719E01382BC90104C080E090E001C0EC
:1023D000CE01DF91CF910895743038F46B3028F43A
:1023E000462F672F0E94D921089580E090E008953C
:1023F0000E94EC110E94E71008958238910569F15E
:10240000B0F48133910509F475C048F4893291051F
:1024100009F467C08A32910509F471C008958533C3
:10242000910509F459C089339105B9F00895833EA7
:10243000910589F138F4803E9105D1F0823E9105F5
:1024400029F10895863E9105C9F1873E9105D9F19C
:10245000843E910509F06CC027C02091B50220FD93
:1024600057C021FD55C02091B60223FD5BC00895E1
:102470008091B50280FD48C08091B60280FF48C0BF
:102480008091B50284FD46C083EE51C08091B502B3
:1024900082FF3CC0F5CF8091B50282FD37C08091AC
:1024A000B60280FD35C0ECCF8091B60281FF36C008
:1024B0008091B50284FD2EC087EE39C08091B502AF
:1024C00083FF2AC0F5CF8091B50283FD25C080919E
:1024D000B60281FD23C0ECCF8091B50285FD22C0FC
:1024E0001FC08091B50285FD1BC08091B60283FF9D
:1024F00019C00AC08091B50286FD16C017C0809130
:10250000B50286FD13C010C089E311C082EE0FC072
:1025100080EE0DC080E00BC086EE09C084EE07C0DF
:1025200085E305C089E203C08AE201C081E390E04F
:1025300008959091B50292FF0DC0282F2871283080
:1025400019F4877F846006C0282F2471243011F489
:102550008B7F886093FF0DC0282F2871283119F4D4
:10256000877E846106C0282F2471243111F48B7E6C
:1025700088612091B60220FF0DC0382F38713830A5
:1025800019F4877F816006C0382F3171313011F422
:102590008E7F886021FF0DC0282F2871283119F403
:1025A000877E816106C0282F2171213111F48E7E32
:1025B000886194FD877E089580E008950E94510F00
:1025C00008950E94E7138FE39CE90197F1F700C09B
:1025D00000000E94E71380E00E94131380FF04C0F4
:1025E0000E94DE120E944E2508950E94E112089575
:1025F0000E94580F811102C00E94EB0F0E94640FCD
:10260000809368020E946E0F9093B6028093B50289
:102610000E94F5120E94690F0E94F909809104023C
:102620000E940E0A0895E82FF0E0EE0FFF1FE1541C
:10263000FD4F808191810895089580EA8A95F1F790
:10264000089500C008950E941D13089508950E94E2
:10265000261308950E94271308950E9426130895B3
:102660000E942D130895F894E82FE295EF70F0E0A2
:1026700031A1282F2F7081E090E001C0880F2A95AA
:10268000EAF7982F9095932391A392A1892B82A387
:10269000789408950F931F93CF93DF93C7E9D1E008
:1026A00089918F3F11F00E94331381E0CB39D80715
:1026B000B9F7CCE8D1E007E911E089918F3F11F03B
:1026C0000E9433130C171D07C1F7DF91CF911F91A3
:1026D0000F910895A0E0B0E0E0E7F3E10C94E02C66
:1026E0008C01C62FD0E0CE0189569E4F6C01FC01B3
:1026F00090819F3F09F450C0B62EF894E92FE295DF
:10270000EF70F0E081A19F7021E030E001C0220F66
:102710009A95EAF7822B81A382A12095282322A3F0
:1027200078940E942113ECE8F1E047E951E021E0C0
:1027300030E0E12CF12C61916F3F89F0A62FA2953A
:10274000AF70B0E090968C9190E06F7002C095955C
:1027500087956A95E2F780FD02C0C90102C080E05A
:1027600090E0E82AF92A220F331F4E175F0719F766
:10277000F60180818F3F11F00E94331361E0E11474
:10278000F10409F460E08B2D0E942313CC0FDD1FB0
:10279000C00FD11FF982E882CDB7DEB7E9E00C9413
:1027A000FC2C0E944A1388E0EFEBF2E0DF01982F47
:1027B0001D929A95E9F7E7EBF2E0DF011D928A9509
:1027C000E9F784E00E9422140E94E2040895A8E040
:1027D000B0E0EDEEF3E10C94E42C8E010F5F1F4F9F
:1027E00088E0F80111928A95E9F7F12C6F2DC80164
:1027F0000E946A13F394F4E0FF12F8CF48E050E02F
:10280000B80187EB92E00E94792D21E0009709F44E
:1028100020E0892B41F088E0F801A7EBB2E00190BD
:102820000D928A95E1F744E06FEB72E087EB92E05E
:102830000E942314182F0E94E504812F2896E5E0BA
:102840000C94002D0895EF92FF920F931F93CF9356
:10285000DF937C018B01C42F222349F081E0809318
:102860006B020E94012590936A0280936902809115
:102870006B02811102C080E01CC0809169029091BE
:102880006A020E9419250597B0F3D0E0CC0FDD1F36
:10289000AE01B701C8010E94792D892B39F0AE0134
:1028A000B701C8010E94862D81E001C080E010922E
:1028B0006B02CDB7DEB7E6E00C94FF2C0E94D62663
:1028C0000E9445100E94E32608950E94E8260E9477
:1028D00054100E94022708950E949E240E94BC2644
:1028E0000E9432100E945E140E9465140E943B10E8
:1028F000FBCFEF92FF920F931F93CF93DF93E82FBD
:1029000071110AC0442321F0F0E0E454FC4FE4913B
:102910006E2F7E2F8E2F6CC0C62FD0E0072F10E0B9
:10292000282F30E0442329F0F901E454FC4F24918E
:1029300030E0CE0166E070E00E943C2CEE24EA9488
:10294000F12CB7010E94802CDB01CC0FDD1FCB01E5
:102950006BEA7FEF0E943C2C8C0F9D1FC82FCC0F81
:10296000C80FC701801B910BB9010E943C2CE92FB5
:10297000492FD0E0CE01B8010E943C2C692F70E0B5
:10298000C701861B970BB9010E943C2CF92FC70188
:102990008C1B9D0BB8010E943C2C692F70E0C70175
:1029A000861B970BB9010E943C2CA230B10591F017
:1029B00038F4109759F01197C1F48E2F7F2F0CC067
:1029C000A430B10579F050F0169779F4722F842F66
:1029D000E92F0DC0892F7E2FE22F09C0822F7E2F75
:1029E000EF2F05C0822F792F02C0722F8F2F6E2FED
:1029F000CDB7DEB7E6E00C94FF2C41E00E947914DD
:102A0000089508950E94FD140895CF93DF93762FC3
:102A1000E901682F842F0E940215798368838A83D5
:102A2000DF91CF9108958091C702282F269530E03D
:102A30002115310519F48170826005C02B323105F2
:102A400024F0817084658093C702089588E090E047
:102A50000E94972D0895CF92DF92EF92FF926B0123
:102A60007C010E941315B701A60188E090E00E9446
:102A7000B52DFF90EF90DF90CF9008956091C70241
:102A80007091C8028091C9029091CA020E942B15D0
:102A90000895E7ECF2E083E0808311828FEF828378
:102AA0008383148260817181828193810E942B15BE
:102AB00008958091C70280FF02C08695089580E046
:102AC00008958091C702817008959091CB02933050
:102AD00018F49F5F9093CB02882351F06091C70256
:102AE0007091C8028091C9029091CA020E942B1570
:102AF000089581E00E94651508959091CB02992375
:102B000019F091509093CB02882351F06091C70245
:102B10007091C8028091C9029091CA020E942B153F
:102B2000089581E00E947D1508958091CB0208955B
:102B30008093CB02662351F06091C7027091C80266
:102B40008091C9029091CA020E942B15089560E0FD
:102B50000E94981508958091C80208958091C90235
:102B600008958091CA02089570E00E943F1C089564
:102B700030910A018091C70280FF0DC08091090148
:102B800090E063E070E00E943C2C632F84539D4FE3
:102B90000E94B415089520910B0140910C01241757
:102BA00068F7822F90E063E070E00E943C2CFC010B
:102BB000E453FD4F1182108212822F5FF0CFA82FB5
:102BC000B62F8091C70280FF16C020910B01309173
:102BD0000C01231770F4822F90E063E070E00E94F4
:102BE0003C2CFC01E453FD4FA183B08342832F5F53
:102BF000F0CF0E94B8150895A3E0B0E0E2E0F6E15E
:102C00000C94E72C9091C70290FF0AC09E012F5FA1
:102C10003F4F0E9405154B8169818A810E94DF1513
:102C20002396E2E00C94032DCF93DF93EC01EC812B
:102C3000F0E0E954FD4F4491E7ECF2E062818181DC
:102C40000E94FC158C818F5F8C83DF91CF9108955A
:102C5000CF93DF93EC01E7ECF2E0438162818C815A
:102C60000E94FC158C818F5F8C83DF91CF9108953A
:102C7000A3E0B0E0EEE3F6E10C94E52C8C0180914A
:102C80006C0281110AC09E012F5F3F4F4FEF6FEF23
:102C90000E9405158A8180936C02F801848181303D
:102CA00051F028F0823061F440916C020AC08091AA
:102CB0006C0240E007C060916C0240E080E003C01D
:102CC00040E080E060E00E94DF15F801848190E040
:102CD000019663E070E00E94942C84832396E4E0E4
:102CE0000C94012DA3E0B0E0E8E7F6E10C94DF2CB2
:102CF000F82ED62EE42EC22E9091C70290FF6EC001
:102D0000E92FE695AE2FB0E0A556BE4F8C9180938B
:102D100096029E7F923061F49E012F5F3F4F8F2D70
:102D20000E9405154B8169818A810E94DF1544C08C
:102D3000823019F4E090CA023FC0863019F4F09056
:102D4000C8023AC08930D9F38931B1F5E9514E2F23
:102D50004170B42EE695F0E0E954FC4FE491A12CCB
:102D60000E2F10E040910D01A41620F52A2D30E021
:102D7000C901B8010E943C2C642F70E00E94802C95
:102D8000EF2DB11002C0E60F01C0E61B80910B01D0
:102D9000A901480F511DCA0163E070E00E943C2C5C
:102DA0009C0124533D4F4E2D6D2D8E2F0E940515F5
:102DB000A394D8CF0E94B815F092C802D092C9024D
:102DC000E092CA02CC2051F06091C7027091C80213
:102DD0008091C9029091CA020E942B152396EAE0C5
:102DE0000C94FB2CE7ECF2E09181282F4381628167
:102DF00088E0890F0E947216089581E00E94F21601
:102E00000895E7ECF2E09181282F4381628188EFF9
:102E1000890F0E947216089581E00E94011708959B
:102E2000E7ECF2E0628128E0620F08F46FEF282FF0
:102E3000438181810E947216089581E00E941017DB
:102E40000895E7ECF2E0628128E0621B08F460E09C
:102E5000282F438181810E947216089581E00E948B
:102E600021170895E7ECF2E0438128E0420F08F4CF
:102E70004FEF282F628181810E947216089581E0B0
:102E80000E9432170895E7ECF2E0438128E0421BEC
:102E900008F440E0282F628181810E947216089513
:102EA00081E00E944317089520E00E947216089561
:102EB000EF92FF921F93CF93DF93EC0110E0EE248B
:102EC000EA94F12C30910D01131700F520910B01BC
:102ED000812F90E0820F911D63E070E00E943C2CF6
:102EE000FC01E453FD4F632F70E0C7010E94942C56
:102EF000812F0E94332C9C819F014091CA026091D6
:102F0000C902890F0E9405151F5FDCCF0E94B8150A
:102F10009A818C8190FF02C08F5F01C081508C83A9
:102F2000DF91CF911F91FF90EF900895A0E0B0E066
:102F3000ECE9F7E10C94DF2CFC01828180FF02C0F8
:102F4000DFEF01C0D1E0C0E036E0A32E80910D019B
:102F5000C81708F043C080910B01CC2ED12C9601EC
:102F6000280F311DC90163E070E00E943C2C84539E
:102F70009D4F7C01FC0111821082128204E010E05E
:102F8000B12C80916E028B0D87302CF06A2D0E943F
:102F9000722C892F05C087FF03C090910D01890F06
:102FA000082E000C990BC816D90691F48091CA021C
:102FB00090E0B8010E943C2C959587959595879552
:102FC0009701482F6091C9028091C8020E9405159F
:102FD000BD0E01501109A9F6CF5FB8CF0E94B815F8
:102FE00080916E02D13031F4811102C080910D01C7
:102FF000815007C090E0019660910D0170E00E9441
:10300000942C80936E02CDB7DEB7EAE00C94FB2CD3
:10301000CF9320910B0130910C01231770F4822F74
:1030200090E063E070E00E943C2CFC01E453FD4F13
:103030001182108212822F5FF0CFC0E060910D01EB
:10304000C61790F5EC2FF0E070E0CF010E94942CB1
:1030500090910B01890F20916D02022E000C330B11
:1030600090E063E070E00E943C2CE217F307A4F0CC
:1030700020910801022E000C330B2E173F0764F03D
:103080009C0124533D4F4091CA026091C902809136
:10309000C8020E94051506C0FC01E453FD4F1182D1
:1030A00010821282CF5FCACF0E94B815209107010B
:1030B00080916D02820F80936D0290910801920FB2
:1030C0009093080119165CF4082E000C990B40919E
:1030D0000D0150E041505109841795071CF02195CE
:1030E00020930701CF910895A0E0B0E0EAE7F8E16E
:1030F0000C94D92C8C01FC01C481CC2ED12CE12C58
:10310000F12CA7019601C701B6010E944D2CA70121
:1031100096010E944D2C4B015C0180E290E06C0115
:10312000CC1AD1080D2C000CEE08FF0825E530E084
:1031300040E050E0C501B4010E944D2C2B013C0140
:10314000A7019601C701B6010E944D2CA701960167
:103150000E944D2C9B01AC01280D391D4A1D5B1DA1
:10316000C301B2010E94A82CD22F822F90E02A32F4
:1031700030F025E530E0A901481B590BCA0163E096
:1031800070E00E943C2C97FD019695958795C82F7D
:10319000C095F12C85E5E82EED1A80910D01F81609
:1031A000D0F4F1FC02C0EE2D01C0ED2F20910B01F7
:1031B0008F2D90E0820F911D63E070E00E943C2C07
:1031C0009C0124533D4F4C2F6091C9028E2F0E94C9
:1031D0000515F394E2CF0E94B815F801848181119E
:1031E00002C091E003C0803219F49FEF9093060172
:1031F00090910601890FF8018483CDB7DEB7E0E135
:103200000C94F52C0F931F93CF93DF93EC0100E008
:1032100010E040910D01842F90E0081719072CF55C
:1032200080910B019801280F311DC90163E070E006
:103230000E943C2C9C0124533D4F469550E08C81CC
:10324000041715071CF4882331F002C0811103C054
:103250004091CA0201C040E06091C9028091C80259
:103260000E9405150F5F1F4FD4CF0E94B8158C81A7
:1032700090E00196817099278C83DF91CF911F9107
:103280000F910895A0E0B0E0E8E4F9E10C94DB2CA4
:10329000FC017280648081E08483E7EBF2E084903B
:1032A000E6E3F3E0E491912CAA24AA94B12CE81966
:1032B000EE2EF12C80910D01981608F0A7C0092D73
:1032C00010E022E0271570F0C80165E070E00E9470
:1032D0003C2CFC01E159FD4F8091C8028083809114
:1032E000C9028183C80165E070E00E943C2C611036
:1032F00006C0FC01E159FD4F138212826BC0EC0144
:10330000C159DD4F8B81882321F181508B8390E05F
:103310006FEF70E00E943C2C6C8170E00E94802C6A
:10332000FB01FF27E954FD4FE4918E2F881990E0AF
:103330006FEF70E00E943C2CB7010E94802C20911E
:10334000CA0230E0862F90E0B9010E943C2C9A839B
:1033500041C00E945C2D9C018091CA0286958158D3
:1033600090E062E071E00E943C2CC92ED12C2C151B
:103370003D0584F532E0371588F40E945C2DB501D7
:103380000E94942C88830E945C2D2091C90226956E
:10339000622F70E00E94942C280F2983C80165E0F9
:1033A00070E00E943C2C81599D4FFC0112822091BB
:1033B000CA02243120F0293C18F028EC01C024E195
:1033C000C80165E070E00E943C2CFC01E159FD4F12
:1033D0002483238380910B019801280F311DC9019B
:1033E00063E070E00E943C2C9C0124533D4FC801D7
:1033F00065E070E00E943C2CFC01E159FD4F4281E8
:10340000618180810E940515939454CF0E94B81564
:10341000CDB7DEB7EEE00C94F72CE7ECF2E080815C
:103420008E7F808360817181828193810E942B15C0
:10343000109297020E94B8150895E7ECF2E080819F
:103440008E7F8083109297020E94B8150895109283
:1034500097028091940281110AC081E080939402C6
:103460008091C7028170809393020E941D1A089573
:103470006091C702669570E04BE050E08EE091E00D
:103480000E946C2D892B19F481E0809397020E9491
:10349000012590938E0280938D0208959091C7022A
:1034A00090FF35C09170811102C0926006C08B32CE
:1034B00010F0946502C0880F982B9093C702662382
:1034C00051F06091C7027091C8028091C902909139
:1034D000CA020E942B156091C702669570E04BE00E
:1034E00050E08EE091E00E946C2D892B19F0109233
:1034F000970202C00E94381A81E0809390024091A6
:10350000CA026091C9028091C8020E9454170895AE
:10351000682F9091C702969581E0890F8B3208F051
:1035200081E00E944E1A089581E00E94881A089551
:10353000682F9091C70296958FEF890F09F48AE260
:103540000E944E1A089581E00E94981A089561E041
:103550000E944E1A0895E7ECF2E08081816080833A
:1035600086950E94A71A08958091C70280FF03C024
:103570000E940D1A08950E94AB1A089560E00E94FF
:103580004E1A08958091950281112EC00E94580F05
:10359000811104C00E94EB0F0E9449150E9426155C
:1035A0006093C7027093C8028093C9029093CA02C5
:1035B0006E7F61F40E9449150E9426156093C70230
:1035C0007093C8028093C9029093CA020E94131597
:1035D000109297028091C70280FF03C086950E94D7
:1035E000BE1A81E0809395020895E7ECF2E08081B5
:1035F0008160808386950E94BE1A08958091C702DB
:1036000080FF03C00E941D1A08950E94F51A0895B4
:10361000109294028091930281110E94F51A0E94E7
:10362000381A08950F931F93CF93DF9380919702D9
:10363000882309F491C080919602E091C702E69533
:10364000E81BE0938F02823049F4F0E0ED54FD4F27
:10365000E491CE2FD0E004E116E159C0863049F460
:10366000F0E0E055FD4FE491CE2FD0E008E216E106
:103670004EC0893051F4E695F0E0E355FD4FE491FA
:10368000CE2FD0E008E517E142C08F3051F4E69527
:10369000F0E0E655FD4FE491CE2FD0E006E917E1CA
:1036A00036C0853149F4F0E0E955FD4FE491CE2F65
:1036B000D0E008E018E12BC08831D9F0833239F42A
:1036C000E5EAF2E0C591D49108E316E120C0843226
:1036D000A9F08532C1F48E2F63E00E94662CE92F99
:1036E000F0E0EE55FD4FE491CE2FD0E002E419E179
:1036F0000EC0C8E2D0E004E718E109C0C4EFD1E091
:1037000002E019E104C0C0EDD7E001E015E18091CD
:103710009002882361F0109290020E9401259093FC
:103720008E0280938D0210929202109291020E945A
:103730000125E0918D02F0918E028E1B9F0B8F3F31
:103740009F4750F4EC0FFD1FF0938E02E0938D0223
:103750008DE892E0F8010995DF91CF911F910F91CB
:103760000895882311F0FA0101C0FB01099508951D
:10377000CF93DF93C82FD62F0E9459158C1738F09E
:103780000E9459158D1718F40E94941A03C08C2FAB
:103790000E94A71ADF91CF9108951F93CF93DF93D3
:1037A000FB011281111166C0EC010E94670E82724A
:1037B000FE01E052F847E531F10508F05AC0EA5B36
:1037C000FF4F0C94CA2C0E94B41A54C043EA5AE129
:1037D00064E97AE104C044E95AE163EA7AE10E94CB
:1037E000B11B48C04CE057E16DEF76E1F8CF4DEFEB
:1037F00056E16CE077E1F3CF4EE257E16DE177E11E
:10380000EECF4DE157E16EE277E1E9CF40E557E1D8
:103810006FE377E1E4CF4FE357E160E577E1DFCF96
:1038200041E955E169E775E1DACF49E755E161E939
:1038300075E1D5CF81E015C065E082E017C068E092
:1038400086E014C06EE089E011C064E18FE00EC034
:1038500067E185E10BC088E104C062E289E106C04E
:1038600083E20E94A71A06C06AE285E20E94B81BA2
:1038700001C011E0812FDF91CF911F9108953F9AF0
:1038800028B12F7738B130684FB7F894FC01CB01DD
:1038900063E070E00E943C2C8E0F9F1FE817F90731
:1038A00089F0519168E038B9000000C057FF28B98D
:1038B000550F000000C000C000C028B900C06A95C4
:1038C00091F7ECCF4FBF8FE594E00197F1F700C07F
:1038D0000000089582E290E00E948F2D823281F4F0
:1038E00083E290E00E948F2D823151F484E290E0D7
:1038F0000E948F2D91E0883009F090E0892F01C05F
:1039000080E081700895CF93C82F811102C06FEFBE
:1039100001C062E282E290E00E94A32DC11102C0C8
:103920006FEF01C062E183E290E00E94A32DC1111C
:1039300002C06FEF01C068E084E290E00E94A32D16
:10394000CF910895089585E290E00E948F2D682F11
:1039500070E080E090E008950895CF93C62F0E9414
:10396000AC1C6C2F85E290E00E94A32DCF910895AE
:1039700080E00E94831C60E070E0CB010E94AD1CDF
:103980000E946C210E942E2281E00E94831C0895D7
:103990000E94A21C0E94A31C0E94AC1C0E946A1CD4
:1039A000811102C00E94B81C08950E94FE1A089559
:1039B000CF93FB01C281CC23E9F09C012250374711
:1039C0002031310520F482500E943E220CC0811526
:1039D000F7E79F0751F481E00E94230A43E062E089
:1039E00081E00E94D804C0E018C081309747A9F454
:1039F00082E0F2CF8115E7E79E0711F481E004C071
:103A00008130974749F482E00E942F0A43E062E048
:103A100081E00E94D80401C0C1E08C2FCF910895AD
:103A20002FEFFC012083089580E00895CF93DF936A
:103A3000EC0188818230D9F078F4813021F50E9440
:103A4000B11590E06FEF70E00E943C2C6FEF70E0DA
:103A50000E94802C698317C0833091F0843099F4E0
:103A60000E94AB1589830E94AE158A830CC00E9408
:103A70006115882319F00E94591504C080E002C026
:103A80000E9495158983DF91CF910895CF93DF939D
:103A9000EC018881823001F1A8F4813079F58981C7
:103AA00090E06FEF70E00E943C2C6FEF70E00E949E
:103AB000802CD62F0E94AE15C82F0E94AB154D2F1B
:103AC0006C2F1AC08330A1F08430C1F40E94B1156C
:103AD000482F6A81898110C08981811103C00E94A9
:103AE0001D1A0CC00E94F51A89810E94BE1A06C0D8
:103AF00089810E94A71502C00E945417DF91CF91BF
:103B00000895FC019C012E5F3F4F9081983041F059
:103B1000993051F0973059F4C9010E94461D08951B
:103B2000C9010E94161D08950E943E1508958FEF49
:103B300080830895FC012181223019F40E94811DA7
:103B400008950E94101D0895EF92FF920F931F9306
:103B5000CF93DF93EC01062F0E94141D8111B1C099
:103B6000E8818E2F90E0FC013197E331F10508F0F8
:103B7000A2C0E55AFF4F0C94CA2C19828BE05EC09C
:103B80008981823089F030F4813009F094C00E943C
:103B90000D250CC0833079F0843009F08CC01A8276
:103BA0001B821C821D8289C00E94A31C9A838B8366
:103BB0007C836D8382C07E0110E0812F0E941313ED
:103BC000F701928383831F5FF2E0EF0EF11C143044
:103BD000A1F773C08981823039F0853009F06BC05C
:103BE0008A810E94D51C69C06A817B818C819D81FC
:103BF0000E94D02C0E94AD1C60C04B816A818981DB
:103C00000E9430219C838D8358C02C813D813227B6
:103C1000232732274B816A8189810E9451214DC01F
:103C20000E946C214AC0602FCE010E949A1D45C09F
:103C30000E94E52124C00E94E72199838A833DC028
:103C40006B8170E089819A81AE014C5F5F4F98274C
:103C5000892798270E94EA2130C06B8170E0898112
:103C60009A81AE014C5F5F4F9827892798270E9461
:103C70000D2223C00E942E2220C00E94172189837A
:103C80001CC06B8170E089819A81AE014C5F5F4FEF
:103C90009827892798270E9497210FC06B8170E091
:103CA00089819A81AE014C5F5F4F982789279827B9
:103CB0000E94B92102C08FEF8883602FCE010E943D
:103CC000C025CDB7DEB7E6E00C94FF2CCF93DF9391
:103CD000FC01DB0112968C91882309F4DDC09F0161
:103CE00030572332310508F0D8C0EF010E946E0F23
:103CF0009093B6028093B502FE01E150F047E232A4
:103D0000F10520F4E259FF4F0C94CA2C8091B502C2
:103D10008160AAC08091B6028860B2C08091B5026D
:103D20008260A2C08091B50220C08091B5028860F7
:103D30009BC08091B6021EC08091B6028260A0C076
:103D40008091B502806190C08091B50280628CC084
:103D50008091B502806488C00E949D098091B5025F
:103D6000806882C08091B502886084607DC0809147
:103D7000B6028260816084C08091B5028E7F74C07B
:103D80008091B602877F7CC08091B5028D7F6CC028
:103D90008091B50220C08091B502877F65C0809177
:103DA000B6021EC08091B6028D7F6AC08091B502B6
:103DB0008F7E5AC08091B5028F7D56C08091B5022A
:103DC0008F7B52C00E949D098091B5028F774CC0B5
:103DD0008091B502877F8B7F47C08091B6028D7F2F
:103DE0008E7F4EC08091B50282FB222720F991E0A0
:103DF000922790FB82F990FB83F936C08091B6023E
:103E0000982F909591708E7F892B90FB81F938C007
:103E10008091B50286FB222720F991E0922790FB42
:103E200086F922C00E949D098091B50287FB222756
:103E300020F991E0922790FB87F916C081E001C03C
:103E400080E00E94EE0F1EC08091B50284FB222705
:103E500020F991E0922790FB84F906C08091B50289
:103E6000982F909590FB80F98093B5020BC08091BC
:103E7000B60283FB222720F991E0922790FB83F979
